:020000020000FC
:1000000009C01CC01CC01CC0B8C0B8C0B8C0B8C0B3
:10001000B8C0B8C00FE90DBF05E003BF02E008BFDC
:1000200002E009BF08E007BB02E007B900E104BB3A
:1000300040E0789400E205BF8895FCCF18951895AC
:100040001FB643954837C9F400EC06B93699FECF80
:1000500004B115B12DED31E0021B130BF1E0E8EE18
:100060000F930DD07ED09CD09BD00F91F2E0E8EAA8
:1000700006D072D040E000E006B91FBE1895E00F30
:100080000027F01F0491083D18F001956FD085D02E
:1000900014E69CD05527003019F051E00CD07DD0EB
:1000A0000F2D1AE093D0502311F405D076D00F2DE8
:1000B00002D073D00895003099F00130B9F00230C9
:1000C000D9F00330F9F0043019F1053039F1063078
:1000D00059F1073079F1083099F10930B9F10895F3
:1000E00057D056D055D054D053D008954CD050D07E
:1000F0004FD04ED04DD0089546D045D049D048D0AD
:1001000047D0089540D03FD03ED042D041D008954E
:100110003AD039D038D037D03BD0089534D033D00E
:1001200032D031D030D0089533D02DD02CD02BD038
:100130002AD008952DD02CD026D025D024D00895B3
:1001400027D026D025D01FD01ED0089521D020D072
:100150001FD01ED018D0089516D015D019D013D0A6
:10016000089516D010D014D00ED0089511D00BD011
:100170000AD009D008D00CD0089518951895189574
:10018000189518951895C39A16D0C39814D0089549
:10019000C39A0DD0C3980FD008950DD00CD00895F8
:1001A0001F9315E008D01A95E9F71F91089503D021
:1001B00002D001D008951F932F9315EA20E72A95C6
:1001C000F1F71A95D9F72F911F910895FF1829E09B
:1001D000001F2A9509F40895FF1CF11A18F4F10E76
:1001E0008894F6CF0894F4CFD8D8D9D9DADADBDB03
:1001F000DCDCDDDDDEDEDFDFE0E0E1E1E2E2E3E307
:10020000E4E4E5E5E6E6E7E7E8E8E9E9EAEAEBEB76
:10021000ECECEDEDEDEEEEEFEFF0F0F1F1F2F2F3EC
:10022000F3F4F4F5F5F6F6F7F7F8F8F9F9FAFAFB5E
:10023000FBFCFCFDFDFEFEFFFF00000101020203CE
:1002400003030404050506060707080809090A0A46
:100250000B0B0C0C0D0D0E0E0F0F101011111212B6
:100260001313141415151616171718181919191A27
:100270001A1B1B1C1C1D1D1E1E1F1F20202121229E
:100280002223232424252526262727282829292A0E
:100290002A2B2B2C2C2D2D2E2E2E2F2F3030313182
:1002A0003232333334343500D8D9DADBDBDCDDDE0F
:1002B000DFE0E1E2E3E3E4E5E6E7E8E9EAEAEBECE4
:1002C000EDEEEFF0F1F1F2F3F4F5F6F7F8F9F9FAF3
:1002D000FBFCFDFEFF000001020304050607070802
:1002E000090A0B0C0D0E0F0F101112131415161610
:1002F0001718191A1B1C1D1D1E1F2021222324251F
:1003000025262728292A2B2C2C2D2E2F303132332D
:10031000333435363738393A3B3B3C3D3E3F40413C
:10032000424243444546474849494A4B4C4D4E4F4B
:100330005051515253545556575858595A5B5C5D59
:100340005E5F5F60616263646566676768696A6B68
:100350006C6D6E6E6F707172737475757677787977
:080360007A7B7C7C7D7E7F002E
:00000001FF
